:020000040000FA
:02000000ED28E9
:080008008E00030E8D000B1E9B
:100010000B288B180E280B19142842283C3094000A
:1000200067200B128B10422847208C03031D1A28CF
:1000300004308C0001300C02031D23281C30850085
:10004000120893003E2802300C02031D2C281A309F
:100050008500110893003E2803300C02031D35284B
:1000600016308500100893003E2804300C02031D52
:100070003E280E3085000F0893003E289D204F201B
:100080000B1142280D0E83008E0E0E0E09000B1A66
:1000900008009403031D08000B168B100800861C33
:1000A0005428181854281614181086181814171CD9
:1000B0006028950303195D28080017101610080022
:1000C000161C080017143C309500802008008F0A89
:1000D0000A300F02031D08008F01900A0A30100237
:1000E000031D08009001910A0A301102031D080047
:1000F0009101920A0A301202031D080092010800C1
:100100008F03FF300F02031D080009308F0090039A
:10011000FF301002031D0800093090009103FF30EA
:100120001102031D0800093091009203FF301202F2
:10013000031D080009309200080000301302031D5F
:10014000A528003086000514080001301302031DA5
:10015000AD28E43086000514080002301302031DA8
:10016000B528903086000510080003301302031DE7
:10017000BD28C03086000510080004301302031D9E
:10018000C528643086000510080005301302031DE1
:10019000CD28483086000510080006301302031DE4
:1001A000D5280C3086000510080007301302031D07
:1001B000DD28E03086000514080008301302031D16
:1001C000E528003086000510080009301302031DE1
:1001D0000800603086000510080083128501860142
:1001E000831645308100003085000330860083127D
:1001F000B0308B00850181019201910190018F0146
:10020000930104308C003C309400950096019701D6
:0602100018140A290A2956
:02400E00F23F7F
:00000001FF
